:020000040000FA
:1000000030260020F9020000010300000303000075
:1000100005030000070300000903000000000000C2
:100020000000000000000000000000000B030000C2
:100030000D030000000000000F030000110300008A
:100040001303000013030000E9060000130300007F
:100050001303000013030000130300001303000048
:100060001303000013030000130300001303000038
:100070001303000013030000130300001303000028
:10008000130300001303000013030000A10300008A
:100090001303000013030000130300001303000008
:1000A00013030000130300001303000013030000F8
:1000B0001303000013030000000000000000000014
:1000C00013030000130300001303000013030000D8
:1000D00013030000130300001303000000000000DE
:1000E0000000000000000000000000000000000010
:1000F0000000000000000000000000000000000000
:1001000000000000000000000000000000000000EF
:1001100000000000000000000000000000000000DF
:1001200000000000000000000000000000000000CF
:1001300000000000000000000000000000000000BF
:1001400000000000000000000000000000000000AF
:10015000000000000000000000000000000000009F
:10016000000000000000000000000000000000008F
:10017000000000000000000000000000000000007F
:10018000000000000000000000000000000000006F
:10019000000000000000000000000000000000005F
:1001A000000000000000000000000000000000004F
:1001B000000000000000000000000000000000003F
:1001C000000000000000000000000000000000002F
:1001D000000000000000000000000000000000001F
:1001E000000000000000000000000000000000000F
:1001F00000000000000000000000000000000000FF
:10020000DFF80CD000F0BAF800480047C90C000035
:100210003026002030B4044654E8000F0D4644E870
:100220000053002BF8D1156030BC704730B4044641
:1002300054E8000F40EA010544E80053002BF7D1D1
:10024000156030BC704730B4044654E8000F00EA33
:10025000010544E80053002BF7D1156030BC70470E
:1002600030B4044654E8000F80EA010544E8005326
:10027000002BF7D1156030BC704730B4044654E809
:10028000000F00EB010544E80053002BF7D1156087
:1002900030BC704730B4044654E8000FA0EB0105B1
:1002A00044E80053002BF7D1156030BC704770B4A0
:1002B00004464FF0000054E8006F0D68AE4207BFDF
:1002C00044E80023012044E800630E60002B1CBFBB
:1002D0000020F0E770BC704730B4044654E8000FCB
:1002E00088422CBF451A054644E80053002BF5D13F
:1002F000156030BC7047000006488047064800473C
:10030000FEE7FEE7FEE7FEE7FEE7FEE7FEE7FEE7C5
:10031000FEE7FEE7CD030000010200000048704741
:100320008426000040EA01039B0703D009E008C9C6
:10033000121F08C0042AFAD203E011F8013B00F8AA
:10034000013B521EF9D27047D2B201E000F8012BF6
:10035000491EFBD270470022F6E710B513460A4645
:1003600004461946FFF7F0FF204610BD421C10F866
:10037000011B0029FBD1801A70470000064C074D75
:1003800006E0E06840F0010394E807009847103465
:10039000AC42F6D3FFF738FF2427000044270000C3
:1003A00010B50121080200F075FC02214FF48270A3
:1003B00000F070FC04214FF4847000F06BFCBDE889
:1003C000104008214FF4867000F064BCF0B5B548C9
:1003D0000023021D0178101D01254FF080540629CD
:1003E0000BD11678360708D10678C6F30316032E0C
:1003F00006D0042E04D0052E02D0062907D00EE028
:10040000B4F82463A84FC6F304263E6002E01678D1
:10041000360704D10678C6F30316032E02D0062948
:1004200004D00FE0A24FA14E7E670EE0167836078B
:1004300008D10678C6F30316032E06D0042E04D086
:10044000052E02D0062907D00EE0D4F84462994F59
:10045000C6F342363E6002E01678360704D10678CD
:10046000C6F30316032E02D0062906D011E0924EE1
:10047000376827F0807737600EE01678360708D1A6
:100480000678C6F30316032E06D0042E04D0052EDC
:1004900002D006290AD011E04FF08046C6F80C3190
:1004A000C6F81031834E361F336002E016783607E7
:1004B00004D10678C6F30316032E02D0062905D010
:1004C0000CE07C4F032664373E600AE0167836075E
:1004D00004D10678C6F30316032E02D006290DD0E8
:1004E00014E0764F05263E60744E78363560734EC4
:1004F000083633603F263F1D3E6002E0167836071F
:1005000004D10678C6F30316052E02D0062957D06B
:1005100062E06B4E36686B4F3E60694E361D366842
:100520003F1D3E60664E083636683F1D3E60644E95
:100530000C3636683F1D3E60614E103636683F1DF2
:100540003E605F4E143636683F1D3E605C4E183686
:1005500036685C4F20373E60594E1C3636683F1D6A
:100560003E60574E203636683F1D3E60544E24365E
:1005700036683F1D3E60524E283636683F1D3E604D
:100580004F4E2C3636683F1D3E604D4E3036366835
:100590004C4F40373E604A4E343636683F1D3E6011
:1005A000474E383636683F1D3E60454E3C3636680D
:1005B0003F1D3E60424E403636683F1D3E6002E0C1
:1005C0001678360708D10678C6F30316032E06D030
:1005D000042E04D0052E02D0062907D019E0D4F845
:1005E0005812394A01F04F01116002E011780907F1
:1005F0000FD10078C0F30310032803D0042801D0E2
:10060000052806D131480168C90702D06FF0010101
:100610000160D4F83001062808D1D4F83401062846
:1006200004D12B48016841F480610160224874388C
:10063000016841F470010160BFF34F8FBFF36F8F0A
:100640004FF01021D1F80002002803DBD1F804029A
:10065000002822DA1F4A15601F480468002CFCD0CD
:100660001524C1F800420568002DFCD0C1F80442F1
:1006700001680029FCD0136001680029FCD0BFF399
:100680004F8F0D48F0380168144A01F4E0611143BE
:100690000160BFF34F8F00BFFDE7124910480860AB
:1006A000F0BD0000E00F00F0403501400DF0ADBAA4
:1006B00000C007403C050040FCED00E01056004043
:1006C0000404001020C50040E40E00400004004077
:1006D0003C17004004E5014000E401400400FA0535
:1006E0000090D0039C0000200148006800470000F3
:1006F0001C00002002E008C8121F08C1002AFAD11D
:1007000070477047002001E001C1121F002AFBD191
:100710007047000072B601F069F800BF00F0B4FE47
:100720000028FBD1104C0121208801EB00400FA1D3
:1007300000F0B6FF10480068C00700D000BE208857
:10074000022101EB00400DA100F0AAFFBFF34F8F83
:100750000948E43801680D4A01F4E0611143016081
:10076000BFF34F8F00BFFDE7B40000204661746106
:100770006C206572726F7200F0ED00E05379737453
:10078000656D207265736574000000000400FA0551
:100790000EB500210091CDE901106A4644F2010036
:1007A000FFF7B8FF0EBD00F003B800F009B8000075
:1007B00072B602480168491C01607047240000209D
:1007C00003490868401E086000D162B67047000007
:1007D000240000202DE9F041064608680C46411C23
:1007E0004FF0A0474FF0010506D005FA00F1C7F819
:1007F0000815206800F050FD6068411C02D00021FF
:1008000000F038FD3168A069C1F82405607D227DC3
:1008100031681043C1F86C05D4E900123068C0F8A3
:100820001425C0F80C15207D012815D1A068411CA5
:1008300002D0002100F01EFDE068411C05D085407B
:10084000C7F80855E06800F027FDD4E902123068C7
:10085000C0F80825C0F81015BDE8F0812DE9F04179
:10086000064608680C46411C4FF0A0474FF00105B2
:1008700006D005FA00F1C7F80815206800F016FD4B
:100880006068411C02D0002100F0FDFC3168A069C5
:10089000C1F82405607D217D32680843C2F86C05EB
:1008A000D4E900123068C0F80C15C0F81425207D7A
:1008B000012815D1A068411C02D0002100F0E3FC02
:1008C000E068411C05D08540C7F80855E06800F095
:1008D000EDFCD4E902123068C0F80825C0F8101504
:1008E000BDE8F0812DE9FC410646C0074FF0000548
:1008F0000ED0104F00240122385D009500231146D0
:10090000019500F06FFC641C042CF4D300F036F861
:10091000B0070DD5074E0024361D0022305D03239D
:1009200000951146019500F05DFC641C042CF4D385
:10093000BDE8FC81B425000007490B5C4FF0A041E5
:10094000D1F804250120984020EA0203C1F80835B7
:100950001040C1F80C057047B42500000249085C3E
:10096000012100F0ADBC0000B42500000249085C84
:10097000002100F0A5BC0000B425000010B5002443
:100980002046FFF7EBFF641C042CF9D310BD0000D8
:100990002DE9F0470546861C90460F464FF00109A9
:1009A0000020FFF700FF1B4C20683860D4E90001ED
:1009B000401AA16804F21C47081A0EE001213846CB
:1009C00000F04CFA00F006F90146384600F046FA0D
:1009D000D4E90001401AA168081A401C8642EDD8EB
:1009E000B8F1000F03D0052065F3891002E006205E
:1009F00065F39F50A2682168114004EB8101C86033
:100A00002068304420600020FFF7CFFE4846BDE854
:100A1000F08700000802002030B482680468531C8C
:100A20008360A154D0E901128A4202D330BC00F0A5
:100A3000CEBA30BC70470000034803C8814201D1E0
:100A400001207047002070470802002010B50021E7
:100A5000024800F00EFA80F3100010BD24060020BA
:100A60002DE9FC5F0E008346DDE90C47C6F100006E
:100A700098469246814600D40846012503E000BF0F
:100A800090FBFAF06D1C5045FADAA84500D94546AE
:100A900024B1002E01DB780700D5641EB80702D50B
:100AA000B8F1000F0AD0F80708D13CB1A54205D231
:100AB00020215846641EFFF7AFFFF6E7002E02DA4A
:100AC0004E462D2102E0780703D52B215846FFF72B
:100AD000A3FF07F0030002280BD1B8F1000F08D1E3
:100AE0003CB1A54205D230215846641EFFF794FF61
:100AF000F6E7CDE90047434652463146584601F0F5
:100B0000F1FCBDE8FC9F000070B50D46044600688E
:100B10004FF4887100F059FF4FF49071206800F095
:100B200054FF4FF49271206800F04FFF4FF4A27110
:100B3000206800F04AFF20681249C0F804132068BA
:100B40006907000B40B2090E002806DA00F00F001A
:100B500000F1E02080F8141D03E000F1E02080F8AF
:100B6000001420680121000B40B200F01F029140E8
:100B70004009800000F1E020C0F88012C0F80011A8
:100B800070BD0000100302000246002012689307A7
:100B900002D0530702D47047500714D502F0030067
:100BA000012802D002280CD105E0C2F383100B68A3
:100BB000801C184404E00223086803EB925210449E
:100BC000086001207047086800EB9253C2F3891057
:100BD000401CEEE72DE9FF410026234800F03BF9D9
:100BE0002148001F074600F036F9204C606800904D
:100BF000A56800E000986946284004EB80000C30AE
:100C0000FFF7C2FF0028F5D101AA009901EA050308
:100C100004EB8303491CDB6842F82030401C009140
:100C20000228F2D3019800F0030001280BD002281B
:100C300010D10198032101EB90500099BDF80A6092
:100C400001EB900005E00198BDF80A60C0F3831045
:100C500008440090384600F0FBF808B10098606046
:100C600004B03046BDE8F0812006002008020020D4
:100C700010B5B0F5827F09D10020FFF75DFE044872
:100C80000168491C01604168491C416010BD0000B9
:100C90000000002078B40A4BC21815680024002D0B
:100CA0000BD0D3F804330B4207D0146011680091C5
:100CB0000449496801B070BC084778BC704700001F
:100CC00000300140140000200EB50120FFF70AFE9D
:100CD000002401220220009423461146019400F0D2
:100CE0006FFA00220D20032300941146019400F0B6
:100CF00067FA4FF40041002000F034FD08B1FFF71F
:100D000047FD00F0B3FB1A4A07CA8DE8070002202E
:100D10008DF808001749684600F07EFE08B1FFF71D
:100D200037FD00F061FE14480321008801EB00400C
:100D300012A100F0B5FC1B4D04242E1F4FF4C87700
:100D400001F082F90120FFF711FE2C60642000F011
:100D5000EDF801F079F90120FFF700FE3460384624
:100D600000F0E4F800F090FB0028FBD1E8E7000079
:100D7000A8250000710C0000B40000204C50434F27
:100D80004D502064726976657220757361676520C5
:100D90006578616D706C6520737461727465642E22
:100DA000000000000C0500502DE9F047C7880446FC
:100DB000181D16468946B0FBF7F1B0FBF7F207FBAA
:100DC00012009A193A44D21CB2FBF7F2DDF820A0C7
:100DD00001E02468491E0029FBD13D1A8846B5422E
:100DE00016D818E0BAF1000F05D0211809EB080059
:100DF0002A46091D04E0204409EB08012A46001D8B
:100E0000FFF790FA00202468761BA844B74201D966
:100E1000354600E03D46002EE4D1BDE8F0870000F5
:100E200030B5024659B100F0C9FC0021074C09E079
:100E300004EB810315685B88AB4202D1116000208E
:100E400030BD491C8142F3D3052030BDA0000020F5
:100E5000002100F009B8012100F010B808B56A4679
:100E6000FFF70BFA009808BD08B56A46FFF7EBF9E3
:100E700008BD08B56A46FFF7CDF908BD08B56A4652
:100E8000FFF7D4F9009808BD08B56A46FFF702FAE3
:100E9000009808BD70B5044600252846FFF783FC7E
:100EA00021686268086890420ED9401E0860017887
:100EB000A38AE26801FB0325227A2168101AC0B2D6
:100EC0000A79824200D208710020FFF76EFC2846A2
:100ED00070BD70B505460C460020FFF764FCE8685D
:100EE000A98A201AB0FBF1F12A681068431C13602C
:100EF0000170BDE870400020FFF757BC10B530B15D
:100F0000017A42680368891AC9B21A6006E00E20A5
:100F100010BD03681A68541C1C601170491EC9B2C8
:100F2000F7D2006800210171084610BD2DE9F0419B
:100F3000040007D0044E4FF47A47751C3846A84782
:100F4000641EFAD1BDE8F081A0250000F0B5054689
:100F50000478154889B0164640F82420124A0869DA
:100F6000121DA2F1080742F82400487F38552022BC
:100F70006846FFF7D7F904942878385C48B10EB179
:100F80000A4A00E000226946281D00F00FFF09B060
:100F9000F0BD0EB1064A00E00022694605F10C00E2
:100FA00000F0D6FDF3E700000C000020C123000094
:100FB0000D2200000FB408B50399002904D004AA3B
:100FC00000926A4600F00FF801B05DF814FB10B50E
:100FD00082680446002A05D0D4E9040321689847B2
:100FE0000020A06010BD2DE9FC4791460C00804612
:100FF00076D014F8011B39B125290ED04046FFF7F1
:101000000BFD20780028F4D198F80C00002867D058
:101010004046BDE8FC47FFF7DABF002001222178F7
:101020002B291BD02D2902D0302908D102E040F015
:10103000010001E040F00200641C002AEFD100250D
:101040002A290ED02178A1F130020A2A11D205EB0B
:10105000850201EB4205641C303DF1E740F00400DD
:10106000EAE7D9F800100B1DC9F800300968641CC4
:101070000D44217800232E290BD114F8011FA1F172
:1010800030020A2A05D203EB830201EB4203303B14
:10109000F3E76C290DD068290BD0692921D00BDC2E
:1010A000252918D0582931D063290ED0642915D1AB
:1010B00017E014F8011FECE7702969D0732932D0CA
:1010C00075291BD0782909D120E0D9F80000011D2D
:1010D000C9F8001001784046FFF79EFC641C90E7B9
:1010E0006CE0D9F800100A1DC9F800200968CDE9A4
:1010F00000500A224046FFF7B3FCEFE7D9F8001092
:101100000A1DC9F8002009680A2206E0D9F8001073
:101110000A1DC9F8002009681022CDE90050404698
:1011200001F0E0F9DAE7D9F8001000270A1DC9F844
:1011300000200E68C00705D112E04046761C7F1CD7
:10114000FFF76AFC31780029F7D104E020214046FE
:101150006D1EFFF761FCBD42C0D9002DF6D1BDE781
:101160004EB13046FFF702F9074604E02021404621
:101170006D1EFFF751FCBD4206D9002DF6D103E0EC
:101180004046761CFFF748FC31780029F8D1A5E7E6
:10119000D9F80000011DC9F800100568302140464B
:1011A000FFF73AFC78214046FFF736FC0820002183
:1011B000CDE90001034610222946B0E7BDE8FC87CF
:1011C00070B541EA4201DDE904564FF0A04441EA1E
:1011D000830141EA052104EB800041EA0641C0F8A1
:1011E000001770BD70B541EA4201DDE904564FF0C9
:1011F000A04441EA830141EA052104EB800041EA71
:101200000641C0F8001770BD70B541EA4201DDE942
:1012100004564FF0A04441EA830141EA052104EB62
:10122000800041EA0641C0F8001770BD70B541EA80
:101230004201DDE904564FF0A04441EA830141EA4E
:10124000052104EB800041EA0641C0F8001770BD9B
:101250001CB5002100910B4601220191FFF7D4FF3C
:101260001CBD1CB5002100910B4601220191FFF726
:10127000DDFF1CBD1CB500220B46009211460192F9
:10128000FFF7C2FF1CBD1CB500220B4600921146A1
:101290000192FFF7CBFF1CBD1CB5002100910B464E
:1012A000012201911146FFF7AFFF1CBD1CB50021C3
:1012B00000910B46012201911146FFF7B7FF1CBDBB
:1012C00001224FF0A043824011B1C3F808257047B6
:1012D000C3F80C257047000030B5124B01460020C2
:1012E000D3F81044224609E0157A854205D1401C06
:1012F0000A28F7DB4FF0FF3030BD5268002AF3D1E7
:10130000421CF9D00872D3F810242AB152684A60FE
:10131000D3F81024516030BD0022C3F810144A6085
:1013200030BD000008020020F0B595B01C461546FF
:101330000F4608461A9E00F011FB182109A8FFF776
:101340000AF80E96CDE909540023082203A938466D
:1013500000F019FB05980690BDF81000ADF81C00D0
:10136000BDF81200ADF81E0000208DF82100039892
:10137000082600F00300012802D0022818D032E02D
:1013800003983346850AC0F3C2008DF82000039805
:101390000FA9C0F38314A200384600F0F4FA09A89C
:1013A000009006AB22460FA9284600F033FA1AE057
:1013B0000398840DC0F3C2008DF82000082C01D2E0
:1013C000254600E0082533462A460FA9384600F096
:1013D000DAFA2E44641B09AB06AA29460FA800F0CE
:1013E0006BF9002CEAD1384600F0BEFA15B0F0BD1A
:1013F0007047012000F028BF084810B50178084A5E
:10140000515C19B1001D00F05DFD02E00C3000F0F0
:101410006BFCBDE81040002000F016BF2C0000203F
:101420000800002008B5034A00924023024AFFF753
:101430007BFF08BD05210000080100200A4A0129A0
:1014400002EBC00007D0022907D0032907D00429E6
:1014500007D00020704702207047042070470079B1
:1014600070474079704700004427000010B5FFF72F
:10147000C0FF04210348FFF72FFF024901204872F3
:1014800010BD0000400000202DE9F0478CB0FFF7B0
:10149000D3FA18B100200CB0BDE8F087784C0020DA
:1014A000C4F81804BFF34F8F60680290A5684FF02E
:1014B0000008284004EB800008E02168029881427F
:1014C00001D86160E6E7284004EB80000C3002A9F7
:1014D000FFF75AFB0028F0D103AB029901EA05029D
:1014E00004EB8202491CD26843F82020401C029180
:1014F0000228F2D3039800F00300022802D001284A
:101500004ED0A5E003985022810D8946B2EB905F42
:1015100000D850210E4666F39F5003900831594879
:1015200000F0D3F9070078D000F018FA43460822FB
:1015300003A9384600F02DFA029908F1080A29405B
:10154000681A8000001D864223D94D4D0C3530B1FC
:10155000C2B204EB8101301A90460C3104E02946F6
:10156000F2B2002590462846C6B25346384600F0EF
:1015700010FA0AEB08032DB1324629464FEA07005C
:1015800000F007FA029909F1030001EB90000290C4
:101590003AE004EB81015346324638460C31EFE71E
:1015A0000398C0F38311062900D3062161F3891043
:1015B0000390C0F38310801C8100324800F085F94D
:1015C000070045D000F0CAF94346082203A938466F
:1015D00000F0DFF908F1080800260FE00298434602
:1015E00000EA0501401C04EB810102900422384608
:1015F0000C3100F0CEF908F10408761C0398C0F312
:101600008310B042EAD847B1D4F81054D4F8180483
:1016100068B1384600F0A8F92CE019E0687A012892
:1016200004D12A6828463946126890476D68002D13
:10163000F4D1384600F098F90020FFF7B4F8D4F858
:10164000180408B9029860600020FFF7AEF811E0B6
:10165000D4F8104404E0216820468968884764680B
:10166000002CF8D108480221008801EB004007A1B6
:1016700000F016F8FFF7E0F980F001000BE700003A
:101680000802002074270000B40000204261636B50
:10169000656E647320666C75736865640000000095
:1016A00000231A4600F04EBD08B5012300926A4699
:1016B00000F048FD08BD00002DE9F0470E468046C9
:1016C0001C46924608293ED894F80C9000202073BE
:1016D0001946104600F06CFC0025B54206D218F8F9
:1016E00005201AA12046FFF765FC03E019A120465A
:1016F000FFF760FC6D1C082DEFD317A12046FFF704
:1017000059FC0025B54210D218F80570FEF706FE08
:101710000068C05D10F03E0F01D03A4600E02E2276
:101720000EA12046FFF746FC03E00DA12046FFF77F
:1017300041FC6D1C082DE5D301222146504600F0E6
:1017400019FC84F80C90BDE8F087000020253032A9
:1017500078000000202020007C00000025630000AD
:1017600020000000104810B5FF21816000210160B9
:101770004160C0F81814C0F8141480F820140B4805
:1017800000F0F0F800280DD109480A490A4B401A28
:10179000C108002003E000BF23F82000401C88425D
:1017A000FAD3002010BD00000802002074270000BA
:1017B0007427000044270000A000002002480349CD
:1017C000401AC0087047000074270000442700003A
:1017D00013B56846FFF724FB08B100201CBD024882
:1017E000009950F831001CBD4427000070B508482E
:1017F0000125D0F8104480F8205405E06572216876
:101800002046496888476468002CF7D170BD000005
:10181000080200202DE9FF4781460C9D00200C4660
:101820002F7B2873984616462946184600F0C0FBC1
:10183000072E42D2DFE806F004090F161F2A3600F1
:1018400049462846FFF7B6FB37E049462846226856
:10185000FFF7B0FB31E0D4E9002349462846FFF703
:10186000A9FB2AE0A0680090D4E900234946284655
:10187000FFF7A0FB21E0D4E90201CDE90001D4E9A2
:10188000002349462846FFF795FB16E004F10800BF
:1018900007C88DE80700D4E9002349462846FFF72A
:1018A00089FB0AE004F108000FC88DE80F00D4E9B5
:1018B000002349462846FFF77DFB00222946404683
:1018C00000F058FB2F73BDE8FF872DE9F041858AB2
:1018D00080462D1F4819C01CB0FBF5F0C6B240462B
:1018E000FFF7D8FA041E19D0002020710120607182
:1018F000E58000272546761EC4F800800BE04046B0
:10190000FFF7C8FA60B16179491C6171286005462A
:101910007F1CC0F80080B742F1D32046BDE8F081BB
:10192000204600F002F80020F8E72DE9F041457963
:1019300001466B1E002201E00968521C9A42FBD34B
:101940000F680146002605E038460C68FFF7C1FA2B
:101950002146761CAE42F7D3BDE8F0810121001D7F
:10196000FFF77CBAFFF7CABA10B504460121001D83
:10197000FFF78AFA10F0FF0F04D12046BDE81040AF
:10198000FFF7D3BF10BD38B501240094FFF70CFA60
:1019900038BD38B500240094FFF706FA38BD40582A
:1019A000002800D00120704708B50022425040585E
:1019B000009008BDD0F80403084000D00120704713
:1019C0004058002800D00120704708B5002242503E
:1019D0004058009008BD0121B1EB507F01D101209A
:1019E0007047002070470000084801220260084844
:1019F0000021C0F80011C0F80411C0F80811C0F8A7
:101A00000C11026003490220087070470035014044
:101A100000300140140000202DE9F041324E05460F
:101A2000307810B10820BDE8F081314C71602F4949
:101A3000204600F063F808B11120F4E7012262604B
:101A40002C49002008602B4F2B78083703F00F0338
:101A50003B602B68DF437F0704D1264FC3F300436D
:101A60000C373B60234F2B79203703F003033B6097
:101A7000204F6B79383703F001033B60C4F8000254
:101A80000F23C4F808332F7A0B680860DFF864C0AE
:101A90000CF1040CDCF800E02EF0070E4EEA070E05
:101AA000CCF800E00B602979E1B1012902D00229CC
:101AB00003D100E00421C4F80413D4F8001241F06B
:101AC0000101C4F80012697A0B4B490183F8001434
:101AD0004FF0E0234FF40021C3F88012C3F8001147
:101AE0003270A0E70821E6E714000020A1030000FF
:101AF000003001400035014013E000E070B50D46B4
:101B000000F0C4FA04000FD00020FEF74CFE20794C
:101B100020B10020FEF749FE112070BD0120256094
:101B200020710020FEF741FE002070BD10B500F0CE
:101B3000ADFA002802D000210160017110BD000043
:101B40000149024800F0A8BBB80000200020004076
:101B50002DE9F0410546007916460F4600EB40019D
:101B60002D4A01EBC00102EB810494F82A1011B157
:101B70000820BDE8F081294951F820102868FFF7B6
:101B8000BDFF08B11120F4E739462846FEF722FED2
:101B900066603869206030004FF001062FD03F7F2B
:101BA0004FF48E712868FFF7FFFE4FF4A27128688A
:101BB000FFF7FAFE28681A49C0F8041328684FEAAC
:101BC0004711000B40B2002806DA00F00F0000F1C8
:101BD000E02080F8141D03E000F1E02080F80014FC
:101BE0002868000B40B200F01F0206FA02F140091B
:101BF000800000F1E020C0F88012C0F800112868D1
:101C00000421C0F800150020A061E06184F82900DB
:101C100044F8140FA675ACE7B8000020BC250000FE
:101C2000800002002DE9F047054600790B4600EBE5
:101C3000400101EBC000234901EB8004284600F07D
:101C400043F810B11120BDE8F0874FF00008C4F848
:101C50002080A360626184F828804FF48E76474626
:101C600031462868FFF7A0FE28684FF00109C0F848
:101C700008902146286800F0ABFA606800BBD5F8F0
:101C800000A00EE094F8280008B10F2716E03146B6
:101C90005046FFF784FE0028F4D02146504600F05D
:101CA00097FA216A60698142F1D331462868FFF7CB
:101CB00076FE0028F9D02868C0F80C90C4F814808B
:101CC0003846C0E7B8000020007900EB400101EB86
:101CD000C000044901EB80004069002800D00120C9
:101CE00070470000B80000202DE9F0470446007955
:101CF0004FF0000900EB400101EBC000254901EB6A
:101D000080072068C0F80095786880B12068224973
:101D1000C0F8081320680121000B40B200F01F0238
:101D200091404009800000F1E020C0F88011206857
:101D3000D0F80C25D0F81485D0F80865D0F81055E7
:101D40004FF0FF31C0F81415C0F80C152068C0F82A
:101D50000815C0F81015501C02D01046FFF778FA8D
:101D6000B8F1FF3F02D04046FFF772FA681C02D07C
:101D70002846FFF76DFA701C02D03046FFF768FA6C
:101D80002068FFF7D3FE87F82A90C7F80490BDE8D3
:101D9000F0870000B80000208402020001490248D8
:101DA00000F026BBE4000020002000402DE9F041B7
:101DB0000546164600790F46154A00EBC00102EBB6
:101DC000810494F8201011B10820BDE8F081114978
:101DD00051F820102868FFF791FE08B11120F4E7B0
:101DE00039462846FEF73AFD6660386920601EB124
:101DF000397F2846FEF788FE28680821C0F80015BC
:101E00000020A061E0610121606184F82010DCE71E
:101E1000E4000020C02500002DE9F04704460E46EE
:101E20000079204900EBC00001EB800517463046E1
:101E3000FFF7D1FD30B1204600F036F820B1112077
:101E4000BDE8F0871020FBE76F61AE604FF490763D
:101E5000002731462068FFF7B8FD4FF4AC784146C3
:101E60002068FFF7B2FD2068AA686969C0F84425B8
:101E7000C0F84815206801218160686878B9B146CA
:101E800049462068FFF79CFD064641462068FFF75B
:101E900097FD0643F4D000B10F2700206861384653
:101EA000CEE70000E40000200079054900EBC00007
:101EB00001EB80004069002800D00120704700003D
:101EC000E40000202DE9F04704460079274900EBA3
:101ED000C00001EB800720684FF00009C0F80095B2
:101EE000786880B120682249C0F808132068012171
:101EF000000B40B200F01F0291404009800000F149
:101F0000E020C0F880112068D0F80C25D0F81485A6
:101F1000D0F80865D0F810554FF0FF31C0F80C1517
:101F2000C0F814152068C0F80815C0F81015501C2A
:101F300002D01046FFF795F9B8F1FF3F02D04046B6
:101F4000FFF78FF9681C02D02846FFF78AF9701C4A
:101F500002D03046FFF785F92068FFF7E7FD87F8E4
:101F60002090C7F80490BDE8F0870000E40000204E
:101F70001003020010B50C46017A052908D0407AFA
:101F800038B1084808A102682046FFF713F800E0BE
:101F90001AB106A12046FFF70DF82046BDE8104013
:101FA000FFF715B878000020257300000D0A000027
:101FB00038B5C3880D46044633B114A0009015A26D
:101FC00016A12846FEF7F6FF217A05291CD0607A73
:101FD00048B1A088FFF732FA164951F8202016A11F
:101FE0002846FEF7E7FFA0880021FFF7F1FB034634
:101FF0001049207A143951F8202001B02846BDE854
:1020000030400EA1FEF7D6BF38BD00001B5B306D1F
:10201000000000001B5B313B33316D0025734C6FBA
:1020200067732064726F70706564202825642925A9
:10203000730D0A0078000020257300003C25733ED4
:102040002025733A2000000070B5094C094D032685
:1020500009E02068401E20602888626806EB004086
:1020600005A1FFF721FB20680028F2D170BD000018
:1020700000000020B40000202325642066616C6C01
:1020800020646574656374656400000003498842D8
:1020900001D1034870470020704700000020004035
:1020A0001C00002070B5054688690C4600284FF4D6
:1020B000847128460AD0FFF777FCD5F81805626AC4
:1020C000E1688854606A401C606270BDFFF76CFC78
:1020D000D5F8180570BD1FB501238DF80030CDE986
:1020E0000121D0E90012684690471FBD1FB50123AA
:1020F0008DF800308DF808100192D0E90012684682
:1021000090471FBD70B50D4C0020D2B22070201D2D
:102110000B4D0378EB5C1BB1001DFFF77DFE02E069
:102120000C30FFF77FFD08B1FEF732FB6078002826
:1021300002D021780029FAD070BD000028000020CC
:10214000080000202DE9F84F204D924689460646AA
:102150009846012269461846AF68FEF719FC58B345
:10216000009800210446801C09E000BF00EA070334
:102170005AF8212005EB8303401C491CDA604145D5
:10218000F4D34FEA164AFEF761FC4AEA0041601CAC
:10219000384005EB80003C4005EB8402C160D0680C
:1021A00066F3C50068F3891069F39F2020F00300EF
:1021B000401C20F00400D06095F8200402E000BF2D
:1021C000FFF762F90028FBD1BDE8F88F0802002074
:1021D00070B50C4605464FF48E71FFF7E5FB216A9A
:1021E000A068415C206A401C2062C5F81C1570BDC7
:1021F0001FB500228DF80020029181680191426193
:10220000D0E90012684690471FBD00001FB50A467E
:1022100001788DF8001041680191017A8DF808105D
:10222000C0680390044850F82210001F50F8222084
:10223000684690471FBD00001000002001490120A2
:10224000087070472800002010B588B0044620228E
:102250000E496846FEF766F806200090C01F019000
:10226000029003904FF0EB7006900CB1084A00E02A
:10227000002269460748FEF769FE08B1FEF788FAB2
:102280000448001F447008B010BD0000E0250000A5
:102290003D2200002C0000202DE9FF470C4605469A
:1022A0004FF40071FFF786FB01274FF401780026F9
:1022B00018B34FF4927949462846FFF770FBE0B116
:1022C00049462846FFF770FBC5F8088394F82900B3
:1022D00000B96F6002208DF80000D5F88004C5F8C1
:1022E00080040390A0690290E0680190A661E66115
:1022F000D4E900126846904728E004212846FFF7F9
:1023000059FB18B34FF484712846FFF748FBE8B136
:1023100021462846FFF7C6FE616AA069884215D1AA
:10232000E06938B1E268616AA0612069E6616662CD
:10233000E06008E094F8290000B96F60C5F80883F0
:10234000A661E268616A2046FFF7C5FE4FF48E7809
:1023500041462846FFF723FB78B1206A616988422D
:1023600002D294F8280020B341462846FFF71CFB10
:10237000616911B12046FFF73BFF4FF4A278414657
:102380002846FFF70CFB002818D041462846FFF7E7
:102390000BFB94F8290000B12F60A06900280DD034
:1023A000A661E268616A04B02046BDE8F047FFF725
:1023B00092BE21462846FFF70BFFDEE7BDE8FF8708
:1023C0001FB50A4601788DF8001041680191017A25
:1023D0008DF80810C0680390044850F82210001FC0
:1023E00050F82220684690471FBD000010000020D2
:1023F0002DE9FF410C464FF4927705463946FFF729
:10240000DFFA0026C0B139462846FFF7DEFA02207F
:102410008DF80000D5F88004C5F880040390D5F845
:102420003C058DF80800E0680190A661E661D4E9FA
:1024300000126846904723E04FF4887739462846D3
:10244000FFF7BEFAE0B139462846FFF7BEFAD5F8E5
:102450003C15A069884213D1E06960B1E268D5F803
:10246000000220F02000C5F80002E069A0612069A8
:10247000E661E06001E0A661E2682046FFF736FE13
:102480004FF4A27739462846FFF79AFA60B13946E9
:102490002846FFF79AFAA06930B1A661D5F83C1535
:1024A0002046E268FFF722FE4FF49077394628462F
:1024B000FFF786FA002813D039462846FFF785FA39
:1024C000606900280CD0D5F84C058DF800608DF8B7
:1024D0000800A06801906661D4E900126846904740
:1024E000BDE8FF812DE9F05F8346DDE90A4A9946A0
:1024F00090460D460846012703E000BFB0FBF8F008
:102500007F1C4045FAD2B94500D94F465FEACA70F0
:1025100012D18CB15FEA8A7002D5B9F1000F01D0F7
:10252000202607E0302605E031465846641EFEF7B7
:1025300073FA0CB1A742F7D35FF00106B9F1010FAE
:1025400002D9A9F1010903E0B5FBF6F0404502D339
:1025500006FB08F6F2E7DFF83C9000BFB5FBF6F0AB
:1025600000FB165519F800105846FEF755FAB6FB51
:10257000F8F6002EF2D15FEACA7009D0002C07D01D
:10258000A74205D220215846641EFEF745FAF5E71A
:10259000BDE8F09FC425000000000000000000001E
:1025A0000338FDD87047000003000000020000005F
:1025B00002070000111213140D0E0F10411B000032
:1025C0009D1D0000303132333435363738394142C1
:1025D0004344454625140000F9130000F1130000A0
:1025E000FFFFFFFFFFFFFFFFFFFFFFFFFFFFFFFFFB
:1025F00000000000000000000000D60107010000FC
:102600000040404040404040404041414141414005
:1026100040404040404040404040404040404040BA
:102620004005020202020202020202020202020249
:10263000022020202020202020202002020202024E
:1026400002029090909090901010101010101010A6
:1026500010101010101010101010101002020202B2
:1026600002028888888888880808080808080808F6
:1026700008080808080808080808080802020202F2
:1026800040000000012600007761726E696E6700ED
:1026900064656275670000001B5B313B33306D0081
:1026A0001B5B306D000000001B5B313B33316D0064
:1026B0001B5B313B33326D001B5B313B33336D00B1
:1026C0001B5B313B33346D001B5B313B33356D009D
:1026D0001B5B313B33366D001B5B313B33376D0089
:1026E000696E666F000000006572726F7200000014
:1026F0004C50434F4D5000005052530055415254DE
:1027000000000000554152544500000062616C6CAD
:102710006F632E6C6F675F6D656D706F6F6C00001F
:10272000617070008C27000000000020B8000000DD
:10273000F406000044280000B800002078250000BE
:1027400004070000F026000000000000F82600004A
:1027500000000000FC26000000000000042700002C
:10276000000000000C2700000000000320270000EC
:1027700000000303540000204C00002054000020FF
:1027800048010020B00000201800000000000000F8
:102790000000000000000000000000000000000039
:1027A0000000000000000000000000000000000029
:1027B00000000000000000000000000000200040B9
:1027C000000000000020004000000000D4250000B0
:1027D00000000000000000000000000000000000F9
:1027E00000000000000000000000000000000000E9
:1027F00000000000E826000088260000E026000017
:1028000090260000A026000098260000A8260000C0
:10281000B0260000B8260000C0260000C826000030
:10282000D0260000D82600000090D0030000000051
:102830000000000000000000000000000000000098
:042840000000000094
:0400000500000201F4
:00000001FF
